S1230020000000000000000000000CBD0CBD0CBD00000000000000000000A07F0000000042
S11C00400000004808186FFF000000000000000000021A006901030059EB
S105009901035D
S10700AC00B000B0EC
S10601007E0CB6B8
S12301511E52554E1E06BE4C4953541E06EC4E45571E06445041541E072E474F5355421E21
S1230171081A474F544F1E083D474F20544F1E083D53495A451E0A665448454E1E0C265058
S123019152494E541E093E4C45541E0A42494E5055541E088749461E0C11454E441E0660F7
S12301B152455455524E1E085044494D1E0A88464F521E0B444E4558541E0BB452454D1ED8
S11101D10A8250415553451E0866201E0A42FC
S123021B0D0A150A1552454144591E23001E1E10161E1E1E4552524F5223201E20494E2040
S123023B4C494E45201E863F8D4DCE00B0C60A8D49810026065A26F77E06609145272681CA
S123025B0D272B810A27E8811527E4811327E0914426088C00B027D70920D48C00F727CF97
S123027BA7000820CA8D32CE02268D2620BC861EA700DFAE8D23397EC0037EC0067E029B21
S123029B36B680042B037E066032398D05200A8DE608A600811E26F7398D12CE02BE8DF2D4
S12302BB8D2039000D0A151EFFFFFFFF1EDF38DE3A0909DF3A369638A7009639A70132DE49
S12302DB3839DE3AEE007C003B7C003B3936378DDCBD046EDE510808DF5109EE00A700E7E8
S12302FB018DDF3332398DC53637DE510808DF5109EE00A600E601BD046333328DC439DE31
S123031B2ADF2CDE2E2002DE249C2C27058D040820F739A6007F004208E600087F004CBD97
S123033B09FB8D22A600088D84CE0152DF4A974BDE4A0909A600811E26F9080808BD02ADDE
S123035BBD02DD7E02A6368620BD029232390808A60081442665BD02C8963CD63DCE0000E4
S123037BE901A90008088C003C26F5847F973CD73DDF209620D6217E0444BD05E5BD0CA26A
S123039BBD044D24013981522606E601C14E27BEBD02C880409756489B569756DE55965580
S12303BBD6566D0226037E0444EE00DF3E0808DF40BD02DDBD05EB812827037E08D208BD21
S12303DB04BDBD02C8BD046E4D27037E0AD5DE3E5D27F8E10022F4A601974F2730DE405AC8
S12303FB2709964F08084A26FB20F4DF40BD02DDBD05E5812C26C408BD04BDBD02C8BD0473
S123041B6E4D26C7DE3E5D27C2E10122BEDE4008085A26FB0909DF40BD02DDBD05E581292A
S123043B2699BD02C89640D641BD02DD08BD04630C3981412B0C815A2F0A81302B048139B6
S123045B2F020D390C398D0B9F289E5137369F519E28399F289E5132339F519E2839BD054B
S123047BE5BD03952504BD030139BD08D72501398128260C088D2BBD05E5812926020839B0
S123049BC60D7E06928DD7BD05E5812A2607088DCD8D4120F2812F2608088DC2BD054220D6
S12304BBE639BD05E5812D2608088DD9BD058D2007812B2601088DCDBD05E5812B260808D9
S12304DB8DC3BD05A320F1812D2608088DB7BD05A120E5398D32860FA7005F4F64036604F4
S12304FB240BEB02A901240586027E0692680269016A0026E74D2BF07D004C2A03BD059A4B
S123051BE704A703BD02DD39BD02C84FDE516D012A048D5E86800808DF516D012A048D5205
S123053B8B80974C0909398DDF6D0126096D022605C6087E069286014C680269012B048185
S123055B1126F5A700A603E6046F036F04E002A2012407EB02A9010C20010D690469036473
S123057B0166026A0026E67D004C2A028D04BD02DD393637BD046E8D06BD046333323943EE
S123059B53CB018900398DEABD046ED750974FBD046EDB50994FBD04630C399632D633D05C
S12305BB319230251CDE2EBD0461E001A200251326035D270F088D18811E26FA089C2A26E3
S12305DBE6DE2A0DDF2CBD046E39A600812026030820F739BD08F22405C6077E0692BD0442
S12305FB619730D731DFAC39DE34A60008811E26F9DF36398DD4DF269F28CE01519E2634D7
S123061B0832E600C11E27131127F5088C01DC2712E600C11E26F4080820E2089FAC9F3494
S123063B9E28399E28CE01DD39DE2EDF2ADF2CDF48094F08A7009C4626F94F97309731972D
S123065B42DE30DF328EA045CE021BBD02A68EA045CEA07FDF3A7F0042BD0282CE00B0BDA1
S123067B05E5DFACBD045525037E0740811E27DEBD060FEE006E008EA045BD02B4CE022F2C
S123069BBD02AD4FBD0463BD09E0CE0237BD02AD5F96362706DE36A600E601BD09FBBD02CA
S12306BBB420A2DE2EDF36CE0059DF57CE0069DF53CEA07FDF3ADE2ADF484F0908A7009CE6
S12306DB4626F9CE0103C64EA700085A26FA7E07F3CE022ABD02A6DE34BD05E5811E272C05
S12306FBBD08F2DF34BD05C0DF24DE3436BD05E5811E322605BD0463200408BD08F24FC685
S123071B01BD05A6BD05C0BD03222003BD031A7E0A8201BD0603CE07F3FFA0468EA040BF45
S123073BA0087EC000BD05EFBD05B6240ADE2C9C2A271E8D502017DEACBD05E5811E260A34
S123075BDE2A9C2E27088D1120048D0D8D377E06698D32DE30DF3220F59F28DE2C9E2AC61A
S123077B0208083434A60034085C811E26F79F2A9F48DE2CF707979C2A2707A600A700084E
S123079B20F59E2839DEACBD060FDF4AD6AFD0ADCB04F707CADB2B8600992A91462234D7B5
S12307BB2B972ADE2ADF489C2C270709A600A70020F5DE2C9F289630A700089631A70008E2
S12307DB964BA700089EAC3432A70008811E26F89E2839C60E7E0692DE369C2A26037E06DE
S12307FB607D003627F80808A60008DF34CE0152DF4A974BCE021ADF51DE4AEE006E00DE2F
S123081B36DF20BD0603DE578C00692605C6097E06929636A700089637A70008DF57DE2059
S123083BDF36DE34BD04BDBD05C02405C6077E0692DF3620A3DE578C00592605C60A7E06F5
S123085B920909DF57EE00DF36208DCE01D3BD02ADBD0361DE36A60008E60008BD09FBBD92
S123087B0295810D26F9BD02B47E0A8296342604C60C2020BD0241CE00B0DFACDE34BD03B7
S123089B95252CDF34DEAC8D43241409A600811E2705C6027E0692BD0241CE00B020E8BD13
S12308BB02E808DFACDE34BD05E508812C27CF097F0042811E27B2C6037E06928D19250646
S12308DBBD046E4D2A020D39BD046339BD05E5974C08812D2704097F004CBD05E5BD0455B2
S12308FB240139094F5F0836A600BD045525268030974E3258492518D750974F58492510F7
S123091B5849250CDB50994F2506DB4E890024D6C6027E0692327D004C2703BD059ABD04DC
S123093B630C39DE34BD05E58122261808A600088122275A811E2604C6042034BD0292BD87
S123095B09D020E9811E261409A60008813B2706BD02B47F004208DF367E07F38154262831
S123097BE601C14126220808A60081422705C60B7E069208BD04BDBD046ED0422310BD03E1
S123099B618D325A26F82006BD04BDBD09E0BD05E5812C261008964216C4F810270CBD0317
S12309BB618D1220F1813B2604087E0940811E2793C60620BB3696424C91432604BD02B487
S12309DB4F97423239BD03618DEB86FF974CBD046E4D2A0CBD059A36862DBD02928DD63287
S12309FBBD02C8CE0A387F004EE001A20025057C004E20F5EB01A90036964E260A8C0A4033
S1230A1B27057D004C260A8B307F004CBD02928DA43208088C0A4226CDBD02DD392710036E
S1230A3BE80064000A0001DE34BD03952405C60C7E0692BD05E508813D2704C60620F1BD96
S1230A5B04BD811E26F5BD02E8201CD6499648D02F922EBD09FBBD0361D6479646D04992D7
S1230A7B48BD09FBBD02B4BD06037E07F3DE34BD05E5BD044D24037E0B298040979A489B29
S1230A9B9A979ABD02C8DE996D00261C6D0126186D0226149649A7019648A700A702BD02F6
S1230ABBDDBD05EB81282705C6057E069208BD04BDBD04615D27034D2704C60F20EC8D556D
S1230ADBA600812C261208BD04BDBD04615D27EA4D26E78D40BD04EF4FC602BD0463BD0483
S1230AFBEFA600812926C108D6499648BD05A64FC602BD05A6BD046E914623037E07EE978F
S1230B1B48D749BD05E5812C2604087E0A8A811E26967E0A82BD02C8DE99EE006D002703CE
S1230B3B0820F9E700BD02DD39DE34BD039524037E0A49DF34BD0461DE538C00992605C6DE
S1230B5B107E0692A70008E70008DF53DE34BD05E508813D27037E0A56BD04BDBD02E808CC
S1230B7B815426F2A60008814F26EBBD04BDBD046EDF34DE53A70008E70008DF53DE34A661
S1230B9B00811E26D108DF36DE539636A70008D637E70008DF537E07F3DE34BD03952403A3
S1230BBB7E0A49BD05E5811E26D908DF36CE0069BD04619C53273AA100262EE101262ABD56
S1230BDB0301BD0461E003A2022505DF537E07F3BD046ECB018900BD02C8EE00A700E701ED
S1230BFBBD02DDEE04DF3620E408080808080820C2C6117E0692DE34BD04BD8D17974DBD5B
S1230C1B04BDDF348D4A24037E0A82DE34BD060FEE006E00BD05E508813D2603860039E65E
S1230C3B00813C2613C13D260408860239C13E260408860339860139813E2705C6067E06C0
S1230C5B92C13D260408860539C13C27E4860439964D4848B70C7DCE0C7EBD05A1BD046E87
S1230C7B4D6E00271820122B12200E2B0E20F4260A200F270D2B022A020D390C395D27FB7B
S1230C9B20F75D26F620F236BD7FE58100270ABD7FEB811B26037E06603239868797027E2B
S1050CBB0644E9
S9030000FC
